Archive member included because of file (symbol)

sargow32.lib(ds00274.o)       edimg.obj (GetFileAttributesA@4)
sargow32.lib(ds00281.o)       edimg.obj (GetFileTime@16)
sargow32.lib(ds00144.o)       edimg.obj (FileTimeToSystemTime@8)
sargow32.lib(ds00676.o)       edimg.obj (SystemTimeToFileTime@8)
sargow32.lib(ds00629.o)       edimg.obj (SetFileTime@16)
sargow32.lib(ds00625.o)       edimg.obj (SetFileAttributesA@8)
../z_tools/win32/w32clibc.lib(startup.obj)
                              (mainCRTStartup)
../z_tools/win32/w32clibc.lib(malloc.obj)
                              edimg.obj (malloc)
../z_tools/win32/w32clibc.lib(stdin.obj)
                              ../z_tools/win32/w32clibc.lib(startup.obj) (__stdin)
../z_tools/win32/w32clibc.lib(fwrite.obj)
                              edimg.obj (fwrite)
../z_tools/win32/w32clibc.lib(fputs.obj)
                              edimg.obj (fputs)
../z_tools/win32/w32clibc.lib(fopen.obj)
                              edimg.obj (fopen)
../z_tools/win32/w32clibc.lib(fread.obj)
                              edimg.obj (fread)
../z_tools/win32/w32clibc.lib(exit.obj)
                              edimg.obj (exit)
../z_tools/win32/w32clibc.lib(fclose.obj)
                              edimg.obj (fclose)
../z_tools/win32/w32clibc.lib(remove.obj)
                              edimg.obj (remove)
../z_tools/win32/w32clibc.lib(fputc.obj)
                              edimg.obj (fputc)
../z_tools/win32/w32clibc.lib(free.obj)
                              ../z_tools/win32/w32clibc.lib(fopen.obj) (free)
../z_tools/win32/libmingw.lib(ds00053.o)
                              edimg.obj (CreateFileA@28)
../z_tools/win32/libmingw.lib(ds00027.o)
                              edimg.obj (CloseHandle@4)
../z_tools/win32/libmingw.lib(dh.o)
                              sargow32.lib(ds00274.o) (_head_libkernel32_a)
../z_tools/win32/libmingw.lib(ds00207.o)
                              ../z_tools/win32/w32clibc.lib(startup.obj) (GetCommandLineA@0)
../z_tools/win32/libmingw.lib(ds00342.o)
                              ../z_tools/win32/w32clibc.lib(startup.obj) (GetStdHandle@4)
../z_tools/win32/libmingw.lib(ds00130.o)
                              ../z_tools/win32/w32clibc.lib(startup.obj) (ExitProcess@4)
../z_tools/win32/libmingw.lib(ds00323.o)
                              ../z_tools/win32/w32clibc.lib(malloc.obj) (GetProcessHeap@0)
../z_tools/win32/libmingw.lib(ds00415.o)
                              ../z_tools/win32/w32clibc.lib(malloc.obj) (HeapAlloc@12)
../z_tools/win32/libmingw.lib(ds00724.o)
                              ../z_tools/win32/w32clibc.lib(fwrite.obj) (WriteFile@20)
../z_tools/win32/libmingw.lib(ds00611.o)
                              ../z_tools/win32/w32clibc.lib(fopen.obj) (SetFilePointer@16)
../z_tools/win32/libmingw.lib(ds00535.o)
                              ../z_tools/win32/w32clibc.lib(fread.obj) (ReadFile@20)
../z_tools/win32/libmingw.lib(ds00088.o)
                              ../z_tools/win32/w32clibc.lib(remove.obj) (DeleteFileA@4)
../z_tools/win32/libmingw.lib(ds00421.o)
                              ../z_tools/win32/w32clibc.lib(free.obj) (HeapFree@12)
../z_tools/win32/libmingw.lib(dt.o)
                              ../z_tools/win32/libmingw.lib(dh.o) (_libkernel32_a_iname)

Memory Configuration

Name             Origin             Length             Attributes
*default*        0x00000000         0xffffffff

Linker script and memory map

                0x00400000                __image_base__ = 0x400000
                0x00000000                __dll__ = 0x0
                0x00001000                __section_alignment__ = 0x1000
                0x00000200                __file_alignment__ = 0x200
                0x00000004                __major_os_version__ = 0x4
                0x00000000                __minor_os_version__ = 0x0
                0x00000001                __major_image_version__ = 0x1
                0x00000000                __minor_image_version__ = 0x0
                0x00000004                __major_subsystem_version__ = 0x4
                0x00000000                __minor_subsystem_version__ = 0x0
                0x00000003                __subsystem__ = 0x3
                0x01c00000                __size_of_stack_reserve__ = 0x1c00000
                0x00001000                __size_of_stack_commit__ = 0x1000
                0x00100000                __size_of_heap_reserve__ = 0x100000
                0x00001000                __size_of_heap_commit__ = 0x1000
                0x00000000                __loader_flags__ = 0x0
LOAD edimg.obj
LOAD autodec.obj
LOAD sargow32.lib
LOAD ../z_tools/win32/w32clibc.lib
LOAD ../z_tools/win32/golibc.lib
LOAD ../z_tools/win32/libmingw.lib

.text           0x00401000     0x4a00
 *(.init)
 *(.text)
 .text          0x00401000     0x32ca edimg.obj
                0x00403b73                opt_binout
                0x00402ace                writefile
                0x0040254d                cmd_exe2bin
                0x00403ce8                decode_l2d3
                0x004014f7                optmatch
                0x004030a4                deletefile
                0x00403adc                opt_binin
                0x00403428                test_BPB
                0x00404107                getattrtime
                0x0040179d                cmd_copy
                0x004016d8                autodecomp2
                0x00402597                dir_search
                0x00401959                getnum
                0x00402960                free_cluster
                0x004020b1                cmd_writedata
                0x00403dd8                getnum_l1b
                0x00401e60                cmd_release
                0x00401a31                cmd_create
                0x00402a43                dir_create
                0x004037f4                opt_vsiz
                0x00403ecc                decode_tek0
                0x00402647                readfile
                0x00401cdf                cmd_setattr
                0x00403f99                sar_shifttime
                0x004031c1                exe2bin
                0x00402215                cmd_list
                0x0040187b                cmd_ovrcopy
                0x00402990                resizefile
                0x00403421                test_KHBIOS
                0x00403e3d                getnum_s8
                0x00401d61                cmd_wbinimg
                0x00403c0d                opt_bias
                0x004016b3                tek1_getnum_s7s
                0x00403c8c                getbc0
                0x004032b4                opt_imgin
                0x00401000                main0
                0x004041de                setattrtime
                0x004021e0                setdec
                0x00402441                cmd_copyall
                0x00403c31                getbc
                0x0040379c                bpbfix_sub
                0x00402da6                ovrwritefile
                0x00403147                setattrfile
                0x00403da4                getnum_l1a
                0x004038f1                opt_imgout
                0x00403e6c                getnum_l0a
                0x004014d1                cmdmatch
                0x00403bf5                opt_bpath
                0x0040151e                pathfix
                0x00403e02                getnum_df
                0x00401c91                cmd_delete
                0x00401b61                cmd_ovrcreate
                0x004014b3                errend
 .text          0x004042ca     0x11aa autodec.obj
                0x004042ca                autodecomp
 *fill*         0x00405474        0xc 00
 .text          0x00405480        0x8 ../z_tools/win32/libmingw.lib(ds00274.o)
                0x00405480                GetFileAttributesA@4
 *fill*         0x00405488        0x8 00
 .text          0x00405490        0x8 ../z_tools/win32/libmingw.lib(ds00281.o)
                0x00405490                GetFileTime@16
 *fill*         0x00405498        0x8 00
 .text          0x004054a0        0x8 ../z_tools/win32/libmingw.lib(ds00144.o)
                0x004054a0                FileTimeToSystemTime@8
 *fill*         0x004054a8        0x8 00
 .text          0x004054b0        0x8 ../z_tools/win32/libmingw.lib(ds00676.o)
                0x004054b0                SystemTimeToFileTime@8
 *fill*         0x004054b8        0x8 00
 .text          0x004054c0        0x8 ../z_tools/win32/libmingw.lib(ds00629.o)
                0x004054c0                SetFileTime@16
 *fill*         0x004054c8        0x8 00
 .text          0x004054d0        0x8 ../z_tools/win32/libmingw.lib(ds00625.o)
                0x004054d0                SetFileAttributesA@8
 .text          0x004054d8       0xf3 ../z_tools/win32/w32clibc.lib(startup.obj)
                0x00405589                mainCRTStartup
 .text          0x004055cb       0x15 ../z_tools/win32/w32clibc.lib(malloc.obj)
                0x004055cb                malloc
 .text          0x004055e0       0xb0 ../z_tools/win32/w32clibc.lib(fwrite.obj)
                0x004055e0                fwrite
 .text          0x00405690       0x33 ../z_tools/win32/w32clibc.lib(fputs.obj)
                0x00405690                fputs
 .text          0x004056c3      0x107 ../z_tools/win32/w32clibc.lib(fopen.obj)
                0x004056c3                fopen
 .text          0x004057ca       0xb1 ../z_tools/win32/w32clibc.lib(fread.obj)
                0x004057ca                fread
 .text          0x0040587b        0xb ../z_tools/win32/w32clibc.lib(exit.obj)
                0x0040587b                exit
 .text          0x00405886       0x2d ../z_tools/win32/w32clibc.lib(fclose.obj)
                0x00405886                fclose
 .text          0x004058b3       0x16 ../z_tools/win32/w32clibc.lib(remove.obj)
                0x004058b3                remove
 .text          0x004058c9       0x25 ../z_tools/win32/w32clibc.lib(fputc.obj)
                0x004058c9                fputc
 .text          0x004058ee       0x15 ../z_tools/win32/w32clibc.lib(free.obj)
                0x004058ee                free
 *fill*         0x00405903        0xd 00
 .text          0x00405910        0x8 ../z_tools/win32/libmingw.lib(ds00053.o)
                0x00405910                CreateFileA@28
 *fill*         0x00405918        0x8 00
 .text          0x00405920        0x8 ../z_tools/win32/libmingw.lib(ds00027.o)
                0x00405920                CloseHandle@4
 *fill*         0x00405928        0x8 00
 .text          0x00405930        0x8 ../z_tools/win32/libmingw.lib(ds00207.o)
                0x00405930                GetCommandLineA@0
 *fill*         0x00405938        0x8 00
 .text          0x00405940        0x8 ../z_tools/win32/libmingw.lib(ds00342.o)
                0x00405940                GetStdHandle@4
 *fill*         0x00405948        0x8 00
 .text          0x00405950        0x8 ../z_tools/win32/libmingw.lib(ds00130.o)
                0x00405950                ExitProcess@4
 *fill*         0x00405958        0x8 00
 .text          0x00405960        0x8 ../z_tools/win32/libmingw.lib(ds00323.o)
                0x00405960                GetProcessHeap@0
 *fill*         0x00405968        0x8 00
 .text          0x00405970        0x8 ../z_tools/win32/libmingw.lib(ds00415.o)
                0x00405970                HeapAlloc@12
 *fill*         0x00405978        0x8 00
 .text          0x00405980        0x8 ../z_tools/win32/libmingw.lib(ds00724.o)
                0x00405980                WriteFile@20
 *fill*         0x00405988        0x8 00
 .text          0x00405990        0x8 ../z_tools/win32/libmingw.lib(ds00611.o)
                0x00405990                SetFilePointer@16
 *fill*         0x00405998        0x8 00
 .text          0x004059a0        0x8 ../z_tools/win32/libmingw.lib(ds00535.o)
                0x004059a0                ReadFile@20
 *fill*         0x004059a8        0x8 00
 .text          0x004059b0        0x8 ../z_tools/win32/libmingw.lib(ds00088.o)
                0x004059b0                DeleteFileA@4
 *fill*         0x004059b8        0x8 00
 .text          0x004059c0        0x8 ../z_tools/win32/libmingw.lib(ds00421.o)
                0x004059c0                HeapFree@12
 *fill*         0x004059c8        0x8 00
 *(SORT(.text$*))
 *(.glue_7t)
 *(.glue_7)
                0x004059d0                ___CTOR_LIST__ = .
                0x004059d0                __CTOR_LIST__ = .
                0x004059d0        0x4 LONG 0xffffffff
 *(SORT(.ctors.*))
 *(.ctors)
 *(.ctor)
                0x004059d4        0x4 LONG 0x0
                0x004059d8                ___DTOR_LIST__ = .
                0x004059d8                __DTOR_LIST__ = .
                0x004059d8        0x4 LONG 0xffffffff
 *(SORT(.dtors.*))
 *(.dtors)
 *(.dtor)
                0x004059dc        0x4 LONG 0x0
 *(.fini)
 *(.gcc_exc)
                0x004059e0                etext = .
 *(.gcc_except_table)

.data           0x00406000      0xe00
                0x00406000                __data_start__ = .
 *(.data)
 .data          0x00406000      0xd42 edimg.obj
                0x00406cd8                len_sec
                0x00406ce0                limit_fat
                0x00406cd0                imgbuf0
                0x00406cf4                KHBIOS
                0x00406ce4                alloc0
                0x00406cf8                fat0
                0x00406004                flag
                0x00406cfc                fat1
                0x00406000                len_imgbuf
                0x00406cec                dir0
                0x00406008                _path
                0x00406ce8                fat
                0x00406cdc                len_clu
                0x00406d00                clu0002
                0x00406ccc                filebuf0
                0x00406cf0                BPB
                0x00406cd4                len_filebuf
 *fill*         0x00406d42        0xe 00
 .data          0x00406d50       0x24 ../z_tools/win32/w32clibc.lib(stdin.obj)
                0x00406d68                __stderr
                0x00406d5c                __stdout
                0x00406d50                __stdin
 .data          0x00406d74        0x2 ../z_tools/win32/w32clibc.lib(fwrite.obj)
 *fill*         0x00406d76        0xa 00
 *(.data2)
 *(SORT(.data$*))
                0x00406d80                __data_end__ = .
 *(.data_cygwin_nocopy)

.rdata
 *(.rdata)
 *(SORT(.rdata$*))
 *(.eh_frame)

.pdata
 *(.pdata)

.bss            0x00407000        0x0
                0x00407000                __bss_start__ = .
 *(.bss)
 *(COMMON)
                0x00407000                __bss_end__ = .

.edata
 *(.edata)

/DISCARD/
 *(.debug$S)
 *(.debug$T)
 *(.debug$F)
 *(.drectve)

.idata          0x00407000      0x400
 SORT(*)(.idata$2)
 .idata$2       0x00407000       0x14 ../z_tools/win32/libmingw.lib(dh.o)
                0x00407000                _head_libkernel32_a
 SORT(*)(.idata$3)
                0x00407014        0x4 LONG 0x0
                0x00407018        0x4 LONG 0x0
                0x0040701c        0x4 LONG 0x0
                0x00407020        0x4 LONG 0x0
                0x00407024        0x4 LONG 0x0
 SORT(*)(.idata$4)
 .idata$4       0x00407028        0x4 ../z_tools/win32/libmingw.lib(dh.o)
 .idata$4       0x0040702c        0x4 ../z_tools/win32/libmingw.lib(ds00027.o)
 .idata$4       0x00407030        0x4 ../z_tools/win32/libmingw.lib(ds00053.o)
 .idata$4       0x00407034        0x4 ../z_tools/win32/libmingw.lib(ds00088.o)
 .idata$4       0x00407038        0x4 ../z_tools/win32/libmingw.lib(ds00130.o)
 .idata$4       0x0040703c        0x4 ../z_tools/win32/libmingw.lib(ds00144.o)
 .idata$4       0x00407040        0x4 ../z_tools/win32/libmingw.lib(ds00207.o)
 .idata$4       0x00407044        0x4 ../z_tools/win32/libmingw.lib(ds00274.o)
 .idata$4       0x00407048        0x4 ../z_tools/win32/libmingw.lib(ds00281.o)
 .idata$4       0x0040704c        0x4 ../z_tools/win32/libmingw.lib(ds00323.o)
 .idata$4       0x00407050        0x4 ../z_tools/win32/libmingw.lib(ds00342.o)
 .idata$4       0x00407054        0x4 ../z_tools/win32/libmingw.lib(ds00415.o)
 .idata$4       0x00407058        0x4 ../z_tools/win32/libmingw.lib(ds00421.o)
 .idata$4       0x0040705c        0x4 ../z_tools/win32/libmingw.lib(ds00535.o)
 .idata$4       0x00407060        0x4 ../z_tools/win32/libmingw.lib(ds00611.o)
 .idata$4       0x00407064        0x4 ../z_tools/win32/libmingw.lib(ds00625.o)
 .idata$4       0x00407068        0x4 ../z_tools/win32/libmingw.lib(ds00629.o)
 .idata$4       0x0040706c        0x4 ../z_tools/win32/libmingw.lib(ds00676.o)
 .idata$4       0x00407070        0x4 ../z_tools/win32/libmingw.lib(ds00724.o)
 .idata$4       0x00407074        0x4 ../z_tools/win32/libmingw.lib(dt.o)
 SORT(*)(.idata$5)
 .idata$5       0x00407078        0x4 ../z_tools/win32/libmingw.lib(dh.o)
 .idata$5       0x0040707c        0x4 ../z_tools/win32/libmingw.lib(ds00027.o)
                0x0040707c                _imp__CloseHandle@4
 .idata$5       0x00407080        0x4 ../z_tools/win32/libmingw.lib(ds00053.o)
                0x00407080                _imp__CreateFileA@28
 .idata$5       0x00407084        0x4 ../z_tools/win32/libmingw.lib(ds00088.o)
                0x00407084                _imp__DeleteFileA@4
 .idata$5       0x00407088        0x4 ../z_tools/win32/libmingw.lib(ds00130.o)
                0x00407088                _imp__ExitProcess@4
 .idata$5       0x0040708c        0x4 ../z_tools/win32/libmingw.lib(ds00144.o)
                0x0040708c                _imp__FileTimeToSystemTime@8
 .idata$5       0x00407090        0x4 ../z_tools/win32/libmingw.lib(ds00207.o)
                0x00407090                _imp__GetCommandLineA@0
 .idata$5       0x00407094        0x4 ../z_tools/win32/libmingw.lib(ds00274.o)
                0x00407094                _imp__GetFileAttributesA@4
 .idata$5       0x00407098        0x4 ../z_tools/win32/libmingw.lib(ds00281.o)
                0x00407098                _imp__GetFileTime@16
 .idata$5       0x0040709c        0x4 ../z_tools/win32/libmingw.lib(ds00323.o)
                0x0040709c                _imp__GetProcessHeap@0
 .idata$5       0x004070a0        0x4 ../z_tools/win32/libmingw.lib(ds00342.o)
                0x004070a0                _imp__GetStdHandle@4
 .idata$5       0x004070a4        0x4 ../z_tools/win32/libmingw.lib(ds00415.o)
                0x004070a4                _imp__HeapAlloc@12
 .idata$5       0x004070a8        0x4 ../z_tools/win32/libmingw.lib(ds00421.o)
                0x004070a8                _imp__HeapFree@12
 .idata$5       0x004070ac        0x4 ../z_tools/win32/libmingw.lib(ds00535.o)
                0x004070ac                _imp__ReadFile@20
 .idata$5       0x004070b0        0x4 ../z_tools/win32/libmingw.lib(ds00611.o)
                0x004070b0                _imp__SetFilePointer@16
 .idata$5       0x004070b4        0x4 ../z_tools/win32/libmingw.lib(ds00625.o)
                0x004070b4                _imp__SetFileAttributesA@8
 .idata$5       0x004070b8        0x4 ../z_tools/win32/libmingw.lib(ds00629.o)
                0x004070b8                _imp__SetFileTime@16
 .idata$5       0x004070bc        0x4 ../z_tools/win32/libmingw.lib(ds00676.o)
                0x004070bc                _imp__SystemTimeToFileTime@8
 .idata$5       0x004070c0        0x4 ../z_tools/win32/libmingw.lib(ds00724.o)
                0x004070c0                _imp__WriteFile@20
 .idata$5       0x004070c4        0x4 ../z_tools/win32/libmingw.lib(dt.o)
 SORT(*)(.idata$6)
 .idata$6       0x004070c8        0xe ../z_tools/win32/libmingw.lib(ds00027.o)
 *fill*         0x004070d6        0x2 00
 .idata$6       0x004070d8        0xe ../z_tools/win32/libmingw.lib(ds00053.o)
 *fill*         0x004070e6        0x2 00
 .idata$6       0x004070e8        0xe ../z_tools/win32/libmingw.lib(ds00088.o)
 *fill*         0x004070f6        0x2 00
 .idata$6       0x004070f8        0xe ../z_tools/win32/libmingw.lib(ds00130.o)
 *fill*         0x00407106        0x2 00
 .idata$6       0x00407108       0x18 ../z_tools/win32/libmingw.lib(ds00144.o)
 .idata$6       0x00407120       0x12 ../z_tools/win32/libmingw.lib(ds00207.o)
 *fill*         0x00407132        0x2 00
 .idata$6       0x00407134       0x16 ../z_tools/win32/libmingw.lib(ds00274.o)
 *fill*         0x0040714a        0x2 00
 .idata$6       0x0040714c        0xe ../z_tools/win32/libmingw.lib(ds00281.o)
 *fill*         0x0040715a        0x2 00
 .idata$6       0x0040715c       0x12 ../z_tools/win32/libmingw.lib(ds00323.o)
 *fill*         0x0040716e        0x2 00
 .idata$6       0x00407170       0x10 ../z_tools/win32/libmingw.lib(ds00342.o)
 .idata$6       0x00407180        0xc ../z_tools/win32/libmingw.lib(ds00415.o)
 .idata$6       0x0040718c        0xc ../z_tools/win32/libmingw.lib(ds00421.o)
 .idata$6       0x00407198        0xc ../z_tools/win32/libmingw.lib(ds00535.o)
 .idata$6       0x004071a4       0x12 ../z_tools/win32/libmingw.lib(ds00611.o)
 *fill*         0x004071b6        0x2 00
 .idata$6       0x004071b8       0x16 ../z_tools/win32/libmingw.lib(ds00625.o)
 *fill*         0x004071ce        0x2 00
 .idata$6       0x004071d0        0xe ../z_tools/win32/libmingw.lib(ds00629.o)
 *fill*         0x004071de        0x2 00
 .idata$6       0x004071e0       0x18 ../z_tools/win32/libmingw.lib(ds00676.o)
 .idata$6       0x004071f8        0xc ../z_tools/win32/libmingw.lib(ds00724.o)
 SORT(*)(.idata$7)
 .idata$7       0x00407204        0x4 ../z_tools/win32/libmingw.lib(ds00027.o)
 .idata$7       0x00407208        0x4 ../z_tools/win32/libmingw.lib(ds00053.o)
 .idata$7       0x0040720c        0x4 ../z_tools/win32/libmingw.lib(ds00088.o)
 .idata$7       0x00407210        0x4 ../z_tools/win32/libmingw.lib(ds00130.o)
 .idata$7       0x00407214        0x4 ../z_tools/win32/libmingw.lib(ds00144.o)
 .idata$7       0x00407218        0x4 ../z_tools/win32/libmingw.lib(ds00207.o)
 .idata$7       0x0040721c        0x4 ../z_tools/win32/libmingw.lib(ds00274.o)
 .idata$7       0x00407220        0x4 ../z_tools/win32/libmingw.lib(ds00281.o)
 .idata$7       0x00407224        0x4 ../z_tools/win32/libmingw.lib(ds00323.o)
 .idata$7       0x00407228        0x4 ../z_tools/win32/libmingw.lib(ds00342.o)
 .idata$7       0x0040722c        0x4 ../z_tools/win32/libmingw.lib(ds00415.o)
 .idata$7       0x00407230        0x4 ../z_tools/win32/libmingw.lib(ds00421.o)
 .idata$7       0x00407234        0x4 ../z_tools/win32/libmingw.lib(ds00535.o)
 .idata$7       0x00407238        0x4 ../z_tools/win32/libmingw.lib(ds00611.o)
 .idata$7       0x0040723c        0x4 ../z_tools/win32/libmingw.lib(ds00625.o)
 .idata$7       0x00407240        0x4 ../z_tools/win32/libmingw.lib(ds00629.o)
 .idata$7       0x00407244        0x4 ../z_tools/win32/libmingw.lib(ds00676.o)
 .idata$7       0x00407248        0x4 ../z_tools/win32/libmingw.lib(ds00724.o)
 .idata$7       0x0040724c       0x10 ../z_tools/win32/libmingw.lib(dt.o)
                0x0040724c                _libkernel32_a_iname

.CRT
 *(SORT(.CRT$*))

.endjunk        0x00408000        0x0
                0x00408000                end = .
                0x00408000                _end = .
                0x00408000                __end__ = .

.rsrc
 *(.rsrc)
 *(SORT(.rsrc$*))

.reloc
 *(.reloc)

.stab
 *(.stab)

.stabstr
 *(.stabstr)
OUTPUT(edimg.exe pei-i386)
